:100000000C9434000C9451000C9451000C94510049
:100010000C9451000C9451000C9451000C9451001C
:100020000C9451000C9451000C9451000C946F00EE
:100030000C9451000C9451000C9451000C945100FC
:100040000C9451000C9451000C9451000C945100EC
:100050000C9451000C9451000C9451000C945100DC
:100060000C9451000C94510011241FBECFEFD8E026
:10007000DEBFCDBF13E0A0E0B1E0EAECF4E202C0E5
:1000800005900D92A43CB107D9F724E0A4ECB3E0AD
:1000900001C01D92A132B207E1F70E94190D0C9424
:1000A00063120C9400008FEF8AB988E08BB9089531
:1000B000E1E8F0E0808188608083808184608083D3
:1000C0008081816080838AE698E1909389008093A3
:1000D0008800EFE6F0E080818260808308951F92BF
:1000E0000F920FB60F9211248F939F93809100016E
:1000F000811104C09BB180E289278BB99F918F91B8
:100100000F900FBE0F901F9018951F93CF93DF9302
:10011000182FEB018091E203811109C081E08093E7
:10012000E203888180931904898180931A0488816D
:10013000829586958770D9F08330E9F587E291E062
:100140000E946B0F69E174E084EC93E00E944E0F13
:10015000E4ECF3E001900020E9F73197AF01445C53
:10016000534064EC73E0812F0E94D6081EC080913A
:100170000001811103C064E271E002C06FE071E030
:1001800084EC93E00E944E0FE4ECF3E00190002039
:10019000E9F73197AF01445C534064EC73E0812F81
:1001A0000E94D608812F0E94BE088881809319047E
:1001B000898180931A04DF91CF911F9108950F9345
:1001C0001F93CF93DF938C01EB018091E2038111A8
:1001D00009C081E08093E2038881809319048981BA
:1001E00080931A048881682F6F7170E0762F6627DC
:1001F0009981690F711D829586958770823009F407
:1002000043C0853009F45FC0811180C020E044EE16
:1002100057E061E082E00E949C07811104C086E300
:1002200091E00E946B0F44EE57E0B80182E00E941B
:100230005808882309F464C02FEF85EA9EE0215016
:1002400080409040E1F700C00000809100018111E2
:1002500003C064E271E002C06FE071E084EC93E0FF
:100260000E944E0FE4ECF3E001900020E9F7319793
:10027000AF01445C534064EC73E082E00E94D60816
:1002800082E00E94BE083CC080910001613071058F
:1002900061F4882351F0109200018EE491E00E94F5
:1002A0006B0F9BB188E089270CC0672B49F5813023
:1002B00038F581E0809300018BE591E00E946B0F9F
:1002C00088E08BB91DC08091000181111FC080E0C2
:1002D00090E00E94530E22E832EE47E45CE30E9475
:1002E000B90E0E941D0E2BEC2603A001279F500D76
:1002F0001124CA018659974E9093890080938800F3
:10030000888180931904898180931A04DF91CF91A9
:100310001F910F910895E82FF0E0ED5EFB4F808173
:100320000895E82FF0E0ED5EFB4F60830895E82F1D
:10033000F0E0EE0FFF1FED50FC4F8081918108959A
:10034000E82FF0E0EE0FFF1FE550FC4F8081918118
:100350000895E82FF0E0EE0FFF1FED5FFB4F808167
:1003600091810895E82FF0E0EE0FFF1FE55FFB4F4E
:10037000808191810895E82FF0E0EE0FFF1FED518D
:10038000FC4F808191810895E82FF0E0EE0FFF1F70
:10039000E551FC4F80819181089524B12C6224B9EC
:1003A0002A9A25B1277D25B920E52CBD2A9820EF72
:1003B0002EBD0DB407FEFDCF9EBD0DB407FEFDCFD3
:1003C0008EBD0DB407FEFDCF6EBD0DB407FEFDCF93
:1003D0002A9A81E0089524B12C6224B92A9A25B181
:1003E000277D25B920E52CBD2A982FE02EBD0DB420
:1003F00007FEFDCF9EBD0DB407FEFDCF8EBD0DB433
:1004000007FEFDCF1EBC0DB407FEFDCF8EB52A9AA8
:10041000089524B12C6224B92A9A25B1277D25B9E3
:1004200020E52CBDFB019B01240F351F60EFE21777
:10043000F307A9F02A986EBD0DB407FEFDCF9EBD4F
:100440000DB407FEFDCF8EBD0DB407FEFDCF71913B
:100450007EBD0DB407FEFDCF2A9A0196E8CFCA01F2
:10046000089524B12C6224B92A9A25B1277D25B993
:1004700020E52CBDFB019B01240F351F6FE0E21727
:10048000F307B1F02A986EBD0DB407FEFDCF9EBDF7
:100490000DB407FEFDCF8EBD0DB407FEFDCF1EBC13
:1004A0000DB407FEFDCF7EB571932A9A0196E7CF72
:1004B000CA0108952F923F924F925F926F927F925E
:1004C0008F929F92AF92BF92CF92DF92EF92FF9264
:1004D0000F931F93CF93DF93CDB7DEB728970FB657
:1004E000F894DEBF0FBECDBF282E362E82EA91E0F3
:1004F0000E946B0F622D8BE190E00E94CD01632D75
:100500008AE190E00E94CD0180E090E49093EC03BA
:100510008093EB0380E090E69093E4038093E30301
:100520008DEA91E00E946B0F83EE882E83E0982E77
:100530009BEEA92E93E0B92E2BEF33E038872F8363
:1005400003EF13E023E0C22E24E0D22E3BE0E32EA3
:1005500034E0F32E1A821982412C512C1C821B820A
:10056000612C712C222D30E03E832D83232C312CE5
:10057000AF81B88511961C921E92F80111821082EB
:100580002B813C8121153042B4F58D819E810980FB
:1005900002C0959587950A94E2F783709927823077
:1005A0009105A9F083309105D9F0019739F080E0E9
:1005B00094E08D939C93EFEFF3E01AC0E0E0F8E055
:1005C000AF81B885ED93FC93EFEFF7E011C0E0E069
:1005D000F0E1AF81B885ED93FC93EFEFFFE008C049
:1005E000E0E0F0E2AF81B885ED93FC93EFEFFFE13F
:1005F000D701ED93FC934114F0E25F069CF5C10135
:10060000098002C0959587950A94E2F7837099272F
:1006100082309105A9F083309105D1F0019741F026
:10062000E0E0F4E0D801ED93FC93EFEFF3E017C0C6
:10063000E0E0F8E0D801ED93FC93EFEFF7E00FC0B6
:10064000E0E0F0E1D801ED93FC93EFEFFFE007C0AD
:10065000E0E0F0E2D801ED93FC93EFEFFFE1D6018B
:10066000ED93FC93AF81B8858D919D91B887AF8351
:100670002B813C81280F391F3C832B83D8012D917E
:100680003D918D01420E531E61147104D9F0EF812A
:10069000F885349760817181F501329740815181ED
:1006A000460F571FF50151834083FD013497608148
:1006B0007181F401329740815181460F571FD40157
:1006C0004D935C93F40160817181F2E08F0E911C77
:1006D000D5014C9111965C91B2E0AB0EB11C3F93E9
:1006E0002F939F938F937F936F935F934F937F92FB
:1006F0006F92A6EDB1E0BF93AF930E94550FFFEF4D
:100700006F1A7F0A29813A812E5F3F4F3A832983EE
:1007100032E0C30ED11C42E0E40EF11C0FB6F89497
:10072000DEBF0FBECDBF94E06916710409F020CF83
:1007300028960FB6F894DEBF0FBECDBFDF91CF91E4
:100740001F910F91FF90EF90DF90CF90BF90AF90EF
:100750009F908F907F906F905F904F903F902F90E1
:100760000895682F80E090E80C94CD0180E80C9407
:10077000B103CF93DF93EC01688181E090E00E94A8
:10078000CD01698182E090E00E94CD016A8183E021
:1007900090E00E94CD016B8184E090E0DF91CF91E9
:1007A0000C94CD01CF93DF93EC0181E090E00E94A7
:1007B000EB01888382E090E00E94EB01898383E073
:1007C00090E00E94EB018A8384E090E00E94EB01BC
:1007D0008B83DF91CF910895CF93DF93EC016881F4
:1007E00085E090E00E94CD01698186E090E00E9462
:1007F000CD016A8187E090E00E94CD016B8188E0A5
:1008000090E0DF91CF910C94CD01CF93DF93EC0179
:10081000688189E090E00E94CD0169818AE090E0E2
:100820000E94CD016A818BE090E00E94CD016B8136
:100830008CE090E00E94CD016C818DE090E00E9400
:10084000CD016D818EE090E0DF91CF910C94CD01D0
:10085000CF93DF93EC0168818FE090E00E94CD019F
:10086000698180E190E00E94CD016A8181E190E0A0
:100870000E94CD016B8182E190E0DF91CF910C94D9
:10088000CD0185E190E00C94EB01CF93C82F692F47
:1008900087E190E00E94CD016C2F88E190E0CF913C
:1008A0000C94CD01682F89E190E00C94CD01682F64
:1008B00086E190E00C94CD01CF93DF93EC0181E0D1
:1008C00090E00E94EB01888382E090E00E94EB01BF
:1008D000898383E090E00E94EB018A8384E090E0CA
:1008E0000E94EB018B83DF91CF910895CF93DF932B
:1008F000EC0185E090E00E94EB01888386E090E0C7
:100900000E94EB01898387E090E00E94EB018A83DB
:1009100088E090E00E94EB018B83DF91CF910895F6
:10092000CF93DF93EC0189E090E00E94EB01888394
:100930008AE090E00E94EB0189838BE090E00E94C6
:10094000EB018A838CE090E00E94EB018B838DE0C9
:1009500090E00E94EB018C838EE090E00E94EB011E
:100960008D83DF91CF910895CF93DF93EC018FE0DA
:1009700090E00E94EB01888380E190E00E94EB010F
:10098000898381E190E00E94EB018A8382E190E01B
:100990000E94EB018B83DF91CF9108950F931F93FA
:1009A000CF93DF938B01C82FD0E02496DC2FCC2788
:1009B000CE0106960E94EB01F8018083CE010796D6
:1009C0000E94EB01F8018183CE0108960E94EB01A1
:1009D000F8018283CE0109960E94EB01F80183831E
:1009E000CE010A960E94EB01F8018483CE010B969A
:1009F0000E94EB01F8018583DF91CF911F910F9148
:100A000008950F931F93CF93DF938B01C82FD0E0EE
:100A10002496DC2FCC27FB016081CE0106960E9434
:100A2000CD01F8016181CE0107960E94CD01F80148
:100A30006281CE0108960E94CD01F8016381CE014A
:100A400009960E94CD01F8016481CE010A960E94A8
:100A5000CD01F8016581CE010B96DF91CF911F91F9
:100A60000F910C94CD010F931F93CF93DF938B01C4
:100A7000C82FD0E02496DC2FCC27CE010C960E9404
:100A8000EB01F8018083CE010D960E94EB01F80185
:100A90008183CE010E960E94EB01F8018283CE0184
:100AA0000F960E94EB01F8018383DF91CF911F9194
:100AB0000F9108950F931F93CF93DF938B01C82F4E
:100AC000D0E02496DC2FCC27FB016081CE010C9670
:100AD0000E94CD01F8016181CE010D960E94CD01E9
:100AE000F8016281CE010E960E94CD01F80163816A
:100AF000CE010F96DF91CF911F910F910C94CD01F4
:100B00000F931F93CF93DF938B01C82FD0E02496D0
:100B1000DC2FCC27CE0140960E94EB01F8018083A8
:100B2000CE0141960E94EB01F8018183DF91CF91C4
:100B30001F910F9108950F931F93CF93DF938B0114
:100B4000C82FD0E02496DC2FCC27FB016081CE019A
:100B500040960E94CD01F8016181CE014196DF915E
:100B6000CF911F910F910C94CD011F93CF93DF93E1
:100B7000162F672FC82FD0E02496DC2FCC27CE016C
:100B800042960E94CD01612FCE014396DF91CF9115
:100B90001F910C94CD0190E0982F88278A5E9B4F7F
:100BA0000C94CD0190E0982F88278C5E9B4F0C947D
:100BB000CD0190E0982F88278E5F9B4F0C94EB011E
:100BC00090E0982F88278D5F9B4F0C94EB01CF927C
:100BD000DF92EF92FF920F931F93CF93DF93C82F73
:100BE000D0E02496DC2FCC277E0180E2E80EF11CB9
:100BF000A19600E010E0C7010E94EB01C82ED12CA5
:100C0000DC2CCC24CE010E94EB01C80ED11CC114F7
:100C1000D10461F0C7010E94EB01082F10E0102FF2
:100C20000027CE010E94EB01080F111D0C151D05B8
:100C300011F7C801DF91CF911F910F91FF90EF90B5
:100C4000DF90CF900895CF92DF92EF92FF920F93B3
:100C50001F93CF93DF93C82FD0E02496DC2FCC27AF
:100C60007E0186E2E80EF11CA79600E010E0C701C5
:100C70000E94EB01C82ED12CDC2CCC24CE010E948A
:100C8000EB01C80ED11CC114D10461F0C7010E9450
:100C9000EB01082F10E0102F0027CE010E94EB017E
:100CA000080F111D0C151D0511F7C801DF91CF911B
:100CB0001F910F91FF90EF90DF90CF900895CF920A
:100CC000DF92EF92FF920F931F93CF93DF93E82F62
:100CD000F0E0EE0FFF1FDF01A55FBB4F8D919C91F0
:100CE000DA01A823B923EF01C551DC4FE880F98070
:100CF000CD018E0D9F1DE550FC4FC081D181AD010E
:100D0000420F531FC417D50778F489016B01CA1B22
:100D1000DB0BAE010E940902A8014C1B5D0BB60162
:100D20006C0F7D1FC70101C0A901DF91CF911F91F9
:100D30000F91FF90EF90DF90CF900C9409028F926B
:100D40009F92BF92CF92DF92EF92FF920F931F93E9
:100D5000CF93DF9300D0CDB7DEB7B82E7A0190E005
:100D60000496982E8824640184E2C80ED11CC60122
:100D700069837A830E94EB01082F10E0102F00276F
:100D800085E2880E911CC4010E94EB01080F111D21
:100D90009701A80169817A818B2D0E945F060E0D53
:100DA0001F1D612FC6010E94CD01602FC4010F904D
:100DB0000F90DF91CF911F910F91FF90EF90DF90F7
:100DC000CF90BF909F908F900C94CD01AF92BF9227
:100DD000CF92DF92EF92FF920F931F93CF93DF9307
:100DE000DA01A901E82FF0E0EE0FFF1FEF01CD5F60
:100DF000DB4F888199816B01C822D922EF01CD5147
:100E0000DC4FE880F980C6018E0D9F1DED50FC4F30
:100E1000C081D1819601240F351FC217D30780F4FA
:100E20008A015D01CC19DD09AE01BD010E943102CC
:100E3000A8014C1B5D0BB5016C0F7D1FC70101C0E4
:100E4000BD01DF91CF911F910F91FF90EF90DF9047
:100E5000CF90BF90AF900C9431029F92AF92BF920F
:100E6000CF92DF92EF92FF920F931F93CF93DF9376
:100E7000982E6B017A01082F10E00C5F1F4F102F86
:100E80000027580188E2A80EB11CC5010E94EB01A1
:100E9000C82FD0E0DC2FCC27075D1F4FC8010E9470
:100EA000EB01C80FD11DDF93CF9387EF91E09F93A4
:100EB0008F930E94550F9701A601BE01892D0E94B4
:100EC000E606CE0DDF1D6D2FC5010E94CD010F90EE
:100ED0000F900F900F906C2FC801DF91CF911F9151
:100EE0000F91FF90EF90DF90CF90BF90AF909F90C9
:100EF0000C94CD010F931F93CF93DF93C82F8FE0F6
:100F000092E00E946B0FD0E02496DC2FCC278E015C
:100F10000F5F1F4F60E1C8010E94CD01C8010E9410
:100F2000EB018111FBCF6FEFCE010296DF91CF91E4
:100F30001F910F910C94CD01CF92DF92EF92FF920F
:100F40000F931F93CF93DF93C82F062F6A01122FA1
:100F500088E192E00E946B0F8FEF800FEC2EF12C56
:100F60008530C8F58C2F0E947A07E7012496DC2F84
:100F7000CC27602F612BCE010E94CD01CE010496BB
:100F80008E010B5F1F4FC114D10429F06D2D0E94FB
:100F9000CD016C2D0FC020911704309118042F5FE4
:100FA0003F4F3093180420931704632F0E94CD0104
:100FB00060911704C8010E94CD018E010F5F1F4F81
:100FC00061E0C8010E94CD01C8010E94EB018111BE
:100FD000FBCF11E001C010E0E7012496DC2FCC2705
:100FE000CE010E94EB01082FCE0103960E94EB0177
:100FF0001F920F931F928F9382E292E09F938F93A1
:101000000E94550F0F900F900F900F900F900F9020
:10101000812FDF91CF911F910F91FF90EF90DF9083
:10102000CF9008950F931F93CF93DF93C82F83E43E
:1010300092E00E946B0FD0E02496DC2FCC278E012B
:101040000D5F1F4FC8010E94EB018331D9F4219637
:1010500062E0CE010E94CD01CE010E94EB01811120
:10106000FBCFC8010E94EB011F928F938DE492E0A9
:101070009F938F930E94550F0F900F900F900F909A
:1010800081E005C08BE592E00E946B0F80E0DF916C
:10109000CF911F910F91089590E0982F88278D5F31
:1010A0009B4F0E94EB01873111F481E00895089570
:1010B000EF92FF920F931F93CF93DF93C82F8B0173
:1010C0007A0185E792E00E946B0FF80160816F3F23
:1010D00051F481818F3F99F482818F3F81F4838124
:1010E0008F3F69F40FC061110AC0F801818181113D
:1010F00006C08281811103C08381882319F0E11425
:10110000F10431F48BE592E00E946B0F80E02FC078
:10111000D0E02496DC2FCC27CE010C960E94CD0186
:10112000F8016181CE010D960E94CD01F801628126
:10113000CE010E960E94CD01F8016381CE010F967B
:101140000E94CD016F2DCE0140960E94CD016E2DE3
:10115000CE0141960E94CD01219664E0CE010E940D
:10116000CD01CE010E94EB018111FBCF81E0DF9127
:10117000CF911F910F91FF90EF900895CF93DF9340
:10118000C82F82E792E00E946B0FD0E0DC2FCC27C3
:10119000CF5FDB4F68E0CE010E94CD01CE010E94FF
:1011A000EB018111FBCFDF91CF9108958F929F9238
:1011B000AF92BF92CF92DF92EF92FF921F93CF93A5
:1011C000DF93182F4B017A018DE993E00E946B0F9A
:1011D000812F0E94A0018E159F0520F4812F0E946F
:1011E000A0017C01C12FD0E02496DC2FCC275E012A
:1011F00083E0A80EB11C812F0E94E7056C01C50198
:101200000E94EB018731A9F08C3199F0DF92CF92E7
:101210001F921F9380E892E09F938F930E94550F37
:101220000F900F900F900F900F900F90E12CF12CDA
:1012300003C0CE14DF04F8F2A701B401812F0E948D
:101240009F066E018FEFC81AD80A60E2C6010E949D
:10125000CD01C6010E94EB018111FBCF2296CE0188
:101260000E94EB0184FD0FC0C5010E94EB018111BA
:10127000F6CF88EA92E00E946B0F812F0E947A07D6
:1012800080E090E005C060E1CE010E94CD01C70181
:10129000DF91CF911F91FF90EF90DF90CF90BF90A3
:1012A000AF909F908F900895AF92BF92CF92DF92B0
:1012B000FF920F931F93CF93DF93F82E6B018A0158
:1012C000C82FD0E02496DC2FCC275E0183E0A80E47
:1012D000B11CC5010E94EB01873191F0C5010E944C
:1012E000EB011F928F9386EB92E09F938F930E9466
:1012F000550F0F900F900F900F908FEF9FEF26C01C
:101300008F2D0E9423065C0118161906ECF489EC57
:1013100092E00E946B0FA016B10620F00115110596
:1013200089F001C08501A801B6018F2D0E942D070B
:10133000219660E4CE010E94CD01CE010E94EB0116
:101340008111FBCFC80102C080E090E0DF91CF9116
:101350001F910F91FF90DF90CF90BF90AF900895B5
:101360009F92AF92BF92CF92DF92EF92FF920F9334
:101370001F93CF93DF93982E5B01EA01790181EDF2
:1013800092E00E946B0F892D0E94A0018C179D078F
:1013900028F4892D0E94A0016C0101C06E01F701A3
:1013A0006081611109C08181811106C08281811132
:1013B00003C08381882331F00115110519F0C11490
:1013C000D10429F5DF93CF931F930F93F701838106
:1013D0001F928F9382811F928F9381811F928F938F
:1013E0001F926F931F929F928BED92E09F938F932A
:1013F0000E94550F8BE592E00E946B0F8DB79EB750
:1014000040960FB6F8949EBF0FBE8DBF49C0C92D40
:10141000D0E02496DC2FCC27CE010C960E94CD0183
:10142000F7016181CE010D960E94CD01F701628125
:10143000CE010E960E94CD01F7016381CE010F9679
:101440000E94CD01612FCE0140960E94CD01602FF8
:10145000CE0141960E94CD01A601B501892D0E94C1
:101460009F068E010F5F1F4F60E2C8010E94CD01F1
:10147000C8010E94EB018111FBCF2296CE010E9490
:10148000EB0184FD10C0CE010E94EB0183FFF6CF7B
:1014900087EB93E00E946B0F68E1CE010E94CD01C3
:1014A00080E090E005C060E1CE010E94CD01C60160
:1014B000DF91CF911F910F91FF90EF90DF90CF9030
:1014C000BF90AF909F9008952F923F924F925F925E
:1014D0006F927F928F929F92AF92BF92CF92DF9244
:1014E000EF92FF920F931F93CF93DF93CDB7DEB7A9
:1014F0002A970FB6F894DEBF0FBECDBF782E4B01F2
:101500006A0179011A8709870E942306892B09F449
:101510002BC183E093E00E946B0F872D0E9423066E
:10152000382E692ECD2809F417C1472C512C84E0A0
:10153000480E511C542C4424520198E2A90EB11CAF
:10154000C5010E94EB01082F10E0102F0027620157
:10155000E9E2CE0ED11CC6010E94EB01080F111D5D
:101560006F923F921F930F938FE093E09F938F931F
:101570000E94550FC2010E94EB010F900F900F9037
:101580000F900F900F908770833009F464C08430FF
:1015900009F4ABC0823009F0D0C028E030E0AE01E1
:1015A0004F5F5F4FB801872D0E94E6061801F8E0F3
:1015B0002F0E311C8981F70180838A8181838B8181
:1015C00082838C8183838D8190E0982F88272E8160
:1015D000820F911DE985FA85918380830F8110E048
:1015E000102F00278885080F111D1F930F938FE27E
:1015F00093E09F938F930E94550FE985FA8581812F
:101600008F9380818F9385E493E09F938F930E94C3
:10161000550FF70183811F928F9382811F928F93C1
:1016200081811F928F9380811F928F9388E593E031
:101630009F938F930E94550F9801A401B101872DAC
:101640000E94E6067101E00EF11E6F2DC5010E9499
:10165000CD016E2D41C026E030E0AE014F5F5F4FFF
:10166000B801872D0E94E606180196E0290E311C6C
:101670008981F70180838A8181838B8182838C8138
:1016800083830D8110E0102F00278E81080F111D1C
:1016900082E793E00E946B0FF70183811F928F9383
:1016A00082811F928F9381811F928F9380811F92DD
:1016B0008F9388E593E09F938F930E94550F980135
:1016C000A401B101872D0E94E606200E311E632D74
:1016D000C5010E94CD01622DC6010E94CD010FB649
:1016E000F894DEBF0FBECDBF2AC022E030E0AE01CD
:1016F0004F5F5F4FB801872D0E94E606780192E0A8
:10170000E90EF11C098110E0902F88270A8110E072
:1017100002501109080F191F9801A401B701872D64
:101720000E94E606E00EF11E6F2DC5010E94CD015C
:101730006E2DC6010E94CD0102C000E010E0EFEF67
:101740004E1A5E0A60E4C2010E94CD01C2010E94ED
:10175000EB018111FBCF02C000E010E086E893E0CE
:101760000E946B0FC80102C080E090E02A960FB67D
:10177000F894DEBF0FBECDBFDF91CF911F910F91C7
:10178000FF90EF90DF90CF90BF90AF909F908F90A1
:101790007F906F905F904F903F902F900895CF92E1
:1017A000DF92FF920F931F93CF93DF93F82E6B017D
:1017B000EA0189E993E00E946B0F8F2D0E94A0013E
:1017C0008C179D0728F48F2D0E94A0018C0101C069
:1017D0008E010115110589F41F921F92DF93CF939B
:1017E00085EA93E09F938F930E94550F0F900F907F
:1017F0000F900F900F900F9030C0A801B6018F2D61
:101800000E949F06CF2DD0E02496DC2FCC276E01BE
:101810008FEFC81AD80A60E2C6010E94CD01C60146
:101820000E94EB018111FBCF6E0182E0C80ED11C3A
:101830002396C6010E94EB0184FD12C0CE010E94D6
:10184000EB01C6010E94EB0183FFF3CF83EB93E032
:101850000E946B0F8F2D0E947A0780E090E005C0F8
:1018600060E1C6010E94CD01C801DF91CF911F91B7
:101870000F91FF90DF90CF900895CF92DF92EF927B
:10188000FF920F931F93CF93DF936C017B018A012B
:10189000E9010E94B60365E585E50E945A02C6018A
:1018A0000E940504C7010E942804C8010E94B903D0
:1018B000CE01DF91CF911F910F91FF90EF90DF90BC
:1018C000CF900C94EC03092E000CAA0BBB0B9C01CF
:1018D000AD0184E0220F331F441F551F8A95D1F7B5
:1018E00060E074E284EF90E00E94FB0D215031092A
:1018F0003093C5002093C40088E18093C10086E046
:101900008093C200E0ECF0E080818D7F80830895B9
:101910009091C00095FFFCCF8093C6000895CF93AF
:10192000C82F8A3019F48DE00E94880C8C2F0E94F9
:10193000880C80E090E0CF9108958091C00087FFEF
:10194000FCCF8091C600089580E895E20E94630C68
:1019500081E091E090931E0480931D04089580938C
:10196000BB0084E88093BC008091BC0087FFFCCF63
:1019700008951092B9008CE08093B80084E08093C1
:10198000BC000895CF9394EA9093BC009091BC0062
:1019900097FFFCCF9091B900987F983011F080E0CC
:1019A00015C0C62F880F0E94AF0C8091B900887FA8
:1019B0008831A9F78C2F0E94AF0C8091B900887FE5
:1019C000883269F784E98093BC0081E0CF91089563
:1019D000CF93DF9394EA9093BC009091BC0097FF63
:1019E000FCCF9091B900987F983011F080E01EC034
:1019F000C42FD62F880F0E94AF0C8091B900887F2A
:101A00008831A1F78D2F0E94AF0C8091B900887F9B
:101A1000883261F78C2F0E94AF0C8091B900887FCB
:101A2000883221F784E98093BC0081E0DF91CF9177
:101A30000895AF92BF92CF92DF92FF920F931F93C0
:101A4000CF93DF93CDB7DEB76A970FB6F894DEBFBA
:101A50000FBECDBF86E0E2E1F1E0DE01119601901C
:101A60000D928A95E1F78091180190911901A0914A
:101A70001A01B0911B018B8B9C8BAD8BBE8B80911F
:101A80001C0190911D01A0911E01B0911F018F8733
:101A9000988BA98BBA8B8091200190912101A09104
:101AA0002201B09123018B879C87AD87BE870E945E
:101AB00053000E9458000E94A40C9E01255F3F4FD6
:101AC000AE01415F5F4FBE016D5E7F4FCE0101965B
:101AD0000E943D0C20E044EE57E062E080E00E946E
:101AE0009C07882309F475C020E044EE57E061E0CC
:101AF00081E00E949C07882309F46BC088E6C82E09
:101B000081E0D82E95E8A92E91E0B92E20E044EE90
:101B100057E061E081E00E949C0781E00E9412088A
:101B2000F12CF110F3CF789483E095E00E94EB0163
:101B3000873121F5F89442E050E0BE01675E7F4FA7
:101B400081E00E94540918161906ACF78A8D1F927D
:101B50008F93898D1F928F93DF92CF920E94550FA2
:101B6000BE01675E7F4F81E00E9485000F900F905D
:101B70000F900F900F900F90FF24F3948E01095E49
:101B80001F4F9E01295F3F4F42E050E0BE01675E5C
:101B90007F4F80E00E94640A089719F6F8948A8DB6
:101BA0001F928F93898D1F928F93BF92AF920E9445
:101BB000550FBE01675E7F4FCE0107960E94DF0082
:101BC000FF24F3940F900F900F900F900F900F90B1
:101BD000A8CF8FEF9FEF6A960FB6F894DEBF0FBEC7
:101BE000CDBFDF91CF911F910F91FF90DF90CF90EC
:101BF000BF90AF900895A1E21A2EAA1BBB1BFD0156
:101C00000DC0AA1FBB1FEE1FFF1FA217B307E407DB
:101C1000F50720F0A21BB30BE40BF50B661F771F33
:101C2000881F991F1A9469F7609570958095909513
:101C30009B01AC01BD01CF0108950E94240E689460
:101C4000B1110C94B30E08950E94980E88F09F571E
:101C500098F0B92F9927B751B0F0E1F0660F771FD0
:101C6000881F991F1AF0BA95C9F714C0B13091F0C6
:101C70000E94B20EB1E008950C94B20E672F782F37
:101C80008827B85F39F0B93FCCF38695779567958B
:101C9000B395D9F73EF490958095709561957F4FF7
:101CA0008F4F9F4F0895E89409C097FB3EF490959D
:101CB0008095709561957F4F8F4F9F4F9923A9F025
:101CC000F92F96E9BB279395F695879577956795B4
:101CD000B795F111F8CFFAF4BB0F11F460FF1BC0F8
:101CE0006F5F7F4F8F4F9F4F16C0882311F096E98B
:101CF00011C0772321F09EE8872F762F05C0662339
:101D000071F096E8862F70E060E02AF09A95660FF1
:101D1000771F881FDAF7880F9695879597F90895AA
:101D200057FD9058440F551F59F05F3F71F047958C
:101D3000880F97FB991F61F09F3F79F08795089571
:101D4000121613061406551FF2CF4695F1DF08C090
:101D5000161617061806991FF1CF869571056105AD
:101D600008940895E894BB2766277727CB0197F955
:101D700008950E94CC0E0C943D0F0E942F0F38F056
:101D80000E94360F20F0952311F00C94260F0C942E
:101D90002C0F11240C94B30E0E94900E70F3959F9B
:101DA000C1F3950F50E0551F629FF001729FBB2752
:101DB000F00DB11D639FAA27F00DB11DAA1F649FEE
:101DC0006627B00DA11D661F829F2227B00DA11DA1
:101DD000621F739FB00DA11D621F839FA00D611D27
:101DE000221F749F3327A00D611D231F849F600D48
:101DF000211D822F762F6A2F11249F5750409AF071
:101E0000F1F088234AF0EE0FFF1FBB1F661F771FFC
:101E1000881F91505040A9F79E3F510580F00C94C7
:101E2000260F0C94B30E5F3FE4F3983ED4F38695EF
:101E300077956795B795F795E7959F5FC1F7FE2B67
:101E4000880F911D9695879597F9089597F99F6743
:101E500080E870E060E008959FEF80EC0895002432
:101E60000A941616170618060906089500240A94FF
:101E700012161306140605060895092E0394000C85
:101E800011F4882352F0BB0F40F4BF2B11F460FF14
:101E900004C06F5F7F4F8F4F9F4F0895FB01DC01A0
:101EA00001900D920020E1F70895A0E0B0E0EBE58D
:101EB000FFE00C943C12AE014B5F5F4FFA01619161
:101EC0007191AF0180911D0490911E040E949B0F9F
:101ED000E2E00C9458120F931F93CF93DF93E0919D
:101EE0001D04F0911E04238121FF1BC08C01D0E052
:101EF000C0E0F80181918F0160911D0470911E0472
:101F0000DB011896ED91FC911997882331F0099522
:101F1000892B79F3DFEFCFEFECCF8AE00995892B9E
:101F200019F08FEF9FEF02C08D2F9C2FDF91CF9183
:101F30001F910F910895ABE0B0E0E1EAFFE00C944F
:101F40002C126C017B018A01FC01178216828381AD
:101F500081FFCCC1CE0101963C01F6019381F701CE
:101F600093FD859193FF81917F01882309F4BAC184
:101F7000853239F493FD859193FF81917F018532FC
:101F800029F4B60190E00E949211E7CF912C212C08
:101F9000312CFFE1F315D8F08B3279F038F4803230
:101FA00079F08332A1F4232D20611DC08D3261F0C0
:101FB000803369F4232D216016C0832D8260382E72
:101FC000E32DE4603E2E2AC0F32DF8601DC037FCDF
:101FD0002DC020ED280F2A3040F08E32B9F436FCA7
:101FE00081C1232D2064322E19C036FE06C08AE03E
:101FF000989E200D1124922E11C0EAE02E9E200DF5
:102000001124222EF32DF0623F2E08C08C3621F4CD
:10201000832D8068382E02C0883641F4F70193FD85
:10202000859193FF81917F018111B3CF982F9F7D7F
:102030009554933028F40C5F1F4F9FE399830DC094
:10204000833631F0833771F0833509F059C021C0F0
:10205000F801808189830E5F1F4F88248394912C1F
:10206000530113C02801F2E04F0E511CF801A0806B
:10207000B18036FE03C0692D70E002C06FEF7FEFC4
:10208000C5010E9487114C018201F32DFF773F2E7D
:1020900016C0280122E0420E511CF801A080B18038
:1020A00036FE03C0692D70E002C06FEF7FEFC501FF
:1020B0000E947C114C01F32DF0683F2E820133FC0D
:1020C0001BC0822D90E088169906B0F4B60180E21C
:1020D00090E00E9492112A94F4CFF50137FC85918B
:1020E00037FE81915F01B60190E00E9492112110AC
:1020F0002A9421E0821A91088114910471F7E8C0B2
:10210000843611F0893641F5F80137FE07C0608149
:102110007181828193810C5F1F4F08C06081718142
:10212000072E000C880B990B0E5F1F4FF32DFF76C7
:102130003F2E97FF09C090958095709561957F4FD0
:102140008F4F9F4FF0683F2E2AE030E0A3010E949E
:10215000CE11882E861845C0853731F4232D2F7E69
:10216000B22E2AE030E025C0932D997FB92E8F360C
:10217000C1F018F4883579F0B5C0803719F0883788
:1021800021F0B0C0E92FE061BE2EB4FE0DC0FB2DE2
:10219000F460BF2E09C034FE0AC0292F2660B22E7B
:1021A00006C028E030E005C020E130E002C020E1B8
:1021B00032E0F801B7FE07C06081718182819381AE
:1021C0000C5F1F4F06C06081718180E090E00E5F60
:1021D0001F4FA3010E94CE11882E8618FB2DFF777A
:1021E0003F2E36FE0DC0232D2E7FA22E891458F4CB
:1021F00034FE0BC032FC09C0832D8E7EA82E05C094
:10220000B82CA32C03C0B82C01C0B92CA4FE0FC05D
:10221000FE01E80DF11D8081803321F49A2D997E15
:10222000A92E09C0A2FE06C0B394B39404C08A2D9F
:10223000867809F0B394A3FC11C0A0FE06C0B214C6
:1022400088F4280C922C9B180EC0B21460F4B601CE
:1022500080E290E00E949211B394F7CFB21418F488
:102260002B1802C0982C212CA4FE10C0B60180E3CC
:1022700090E00E949211A2FE17C0A1FC03C088E763
:1022800090E002C088E590E0B6010CC08A2D867807
:1022900059F0A1FE02C08BE201C080E2A7FC8DE2F2
:1022A000B60190E00E949211891438F4B60180E3DF
:1022B00090E00E9492119A94F7CF8A94F301E80D6E
:1022C000F11D8081B60190E00E9492118110F5CF3E
:1022D000222009F442CEB60180E290E00E949211E1
:1022E0002A94F6CFF6018681978102C08FEF9FEF87
:1022F0002B96E2E10C944812FC010590615070406D
:102300000110D8F7809590958E0F9F1F0895FC01BE
:102310006150704001900110D8F7809590958E0F14
:102320009F1F08950F931F93CF93DF93FB0123818A
:1023300021FD03C08FEF9FEF2CC022FF16C0468106
:102340005781248135814217530744F4A081B1811C
:102350009D012F5F3F4F318320838C9326813781EE
:102360002F5F3F4F3783268314C08B01EC01FB01A5
:102370000084F185E02D0995892BE1F6D8011696A8
:102380008D919C911797019617969C938E93169713
:10239000CE01DF91CF911F910F910895FA01AA27E5
:1023A000283051F1203181F1E8946F936E7F6E5F98
:1023B0007F4F8F4F9F4FAF4FB1E03ED0B4E03CD046
:1023C000670F781F891F9A1FA11D680F791F8A1F29
:1023D000911DA11D6A0F711D811D911DA11D20D090
:1023E00009F468943F912AE0269F11243019305D4A
:1023F0003193DEF6CF010895462F4770405D41933B
:10240000B3E00FD0C9F7F6CF462F4F70405D4A3387
:1024100018F0495D31FD4052419302D0A9F7EACF4F
:10242000B4E0A6959795879577956795BA95C9F77E
:1024300000976105710508959B01AC010A2E069471
:102440005795479537952795BA95C9F7620F731F2A
:10245000841F951FA01D08952F923F924F925F9267
:102460006F927F928F929F92AF92BF92CF92DF92A4
:10247000EF92FF920F931F93CF93DF93CDB7DEB709
:10248000CA1BDB0B0FB6F894DEBF0FBECDBF09949D
:102490002A88398848885F846E847D848C849B84F4
:1024A000AA84B984C884DF80EE80FD800C811B8102
:1024B000AA81B981CE0FD11D0FB6F894DEBF0FBE31
:0A24C000CDBFED010895F894FFCFA1
:1024CA000100000002000000008F0C000000002044
:1024DA000000A0BDCDDDEDFDC0A801CDC0A8010161
:1024EA00FFFFFF0020010052657175657374204378
:1024FA006F6D4D656D00534F434B4554204E4F4E03
:10250A0020494E4954494C494153454520004D4FB5
:10251A00444520455645494C4C45004D4F444520BD
:10252A00534F4D4D45494C004D4553534147452066
:10253A00524543552056494120544350202578207E
:10254A002578200A004D45535341474520524543BB
:10255A005520564941205544502025782025782079
:10256A000A00737973696E697428290D00436861DA
:10257A006E6E656C203A2053454E44204D454D20E1
:10258A0053495A45203A2052454356204D454D203D
:10259A0053495A450D002564203A20252E347820C7
:1025AA003A20252E3478203A20252E3478203A20D5
:1025BA00252E34780D0A004953525F52583A207238
:1025CA00645F707472203A20252E34780D0A0063F5
:1025DA006C6F736528290D00736F636B6574282906
:1025EA000D00536E5F5352203D20252E3278202C49
:1025FA002050726F746F636F6C203D20252E3278E5
:10260A000D0A006C697374656E28290D0073746174
:10261A00747573203D2025780D0A004661696C5B4C
:10262A00696E76616C69642069702C706F72745D72
:10263A000D00646973636F6E6E65637428290D00FB
:10264A00736F636B657420256420667265657369B0
:10265A007A652825642920656D707479206F722047
:10266A006572726F720D0A00534F434B5F434C4FB2
:10267A005345442E0D00426164207374617475736E
:10268A00203D20253032780A007265637628290DAC
:10269A000073656E64746F28290D002564204661F5
:1026AA00696C5B252E32782E252E32782E252E3215
:1026BA00782E252E32782C20252E642C2025645D38
:1026CA000D0A007265637666726F6D28290D0049DE
:1026DA0053525F52583A2072645F707472203A20E3
:1026EA00252E34782073697A653D25640D0A0055D4
:1026FA004450206D736720232564206172726976C5
:10270A0065640D0A00736F7572636520506F727489
:10271A00203A2025750D0A00736F7572636520498A
:10272A0050203A2025642E25642E25642E25640D1A
:10273A000A00495020524157206D73672061727216
:10274A00697665640D007265637666726F6D282915
:10275A0020656E64202E2E0D0069676D7073656E9C
:10276A006428290D002564204661696C5B25645D37
:10277A000D0A0069676D7073656E64206661696C25
:04278A002E0D000010
:00000001FF
